:04000000D4EF04F045
:0800080000C504F501C505F572
:1000100002C506F5076A03C508F50001F5C409F530
:10002000F6C40AF5F7C40BF5F8C40CF5A1AE1CEF45
:1000300000F0B1BE2EEF00F009C5F5F40AC5F6F4E4
:100040000BC5F7F40CC5F8F404C500F505C501F5BA
:1000500006C502F5078E08C503F51100000103016E
:100060001AA901D0196B070E186F1C524AE02250D2
:10007000000A00010BE0010A0EE0030A16E0010A83
:100080001EE0070A26E0010A2EE037D01BC57DF0EE
:10009000010E1D6E34D026A805D01BC57DF0010EC3
:1000A0001D6E02D07D6B1D6A2AD026A605D01BC509
:1000B0007DF0010E1D6E02D07D6B1D6A20D026A43E
:1000C00005D01BC57DF0010E1D6E02D07D6B1D6A33
:1000D00016D026A205D01BC57DF0010E1D6E02D0E4
:1000E0007D6B1D6A0CD026A005D01BC57DF0010ECE
:1000F0001D6E02D07D6B1D6A02D07D6B1D6A04D01F
:10010000030100017D6B1D6ACFB61BD0245219E09C
:10011000CFA40CD0235205E11B3C01D001D01B2AF7
:1001200004D02250050801E0222A09D0235204E11C
:100130001B5201E01B0603D0225201E02206246A72
:1001400003D0246ACFB6242ACFB806D0255204E0C3
:10015000010E216E256A03D0256ACFB8252ACFB8B3
:100160000CD01E2AD8B41F2A1E50B80805E11F5013
:100170000B0802E1010E206E03D01F6A1E6A206A7E
:10018000262AB19E1CEF00F04C4F414420465245B8
:100190000000512020204443202000005120202036
:1001A0003632487A0000512020313235487A00003A
:1001B000512020323530487A00005120203530302F
:1001C000487A0000512031303030487A0000454CE8
:1001D000455F4C4F414400002076322031412020C1
:1001E00000004F5645522D562020000025352E3355
:1001F000664120200000204F5645522D4920000026
:1002000025342E3266204F464600050EEA6E300E2B
:10021000E96EEF500EE0140E016E006A002EFED75C
:10022000012EFBD7BF0E006E002EFED700D0EF2EA2
:10023000F2D71200FF0EC66EC76EC86E04010969C0
:10024000C89CC89EC790C792C898C89AA00E0001C3
:100250007F6F080E0301F56FF66B1F0EFA6FEF6BE1
:10026000100EEE6FE76B840EF36F000EF86F030E47
:100270000401006F000E086F106F206F00011DEF6A
:1002800005F03FA802D0C08801D0C0983FA602D098
:10029000BF8201D0BF923FA402D0BF8001D0BF90E7
:1002A0003FA202D0C08E01D0C09E3FA002D0C08C21
:1002B00001D0C09C1200C08A00D0C09A00D01200A9
:1002C000640E306EA2DF030E3F6EDBDFF4DF050E3F
:1002D000306E9BDF030E3F6ED4DFEDDF010E306E1C
:1002E00094DF030E3F6ECDDFE6DF010E306E8DDF53
:1002F000020E3F6EC6DFDFDF010E306E86DF020EBC
:100300003F6EBFDFD8DF010E306E7FDF0E0E3F6E17
:10031000B8DFD1DF010E306E78DF3F6AB2DFCBDFAE
:10032000010E306E72DF080E3F6EABDFC4DF010ED0
:10033000306E6BDF3F6AA5DFBEDF010E306E65DF1A
:100340000C0E3F6E9EDFB7DF010E306E5EDF3F6A40
:1003500098DFB1DF010E306E58DF060E3F6E91DF81
:10036000AADF010E306E51DF3F6A8BDFA4DF010E82
:10037000306E4BDF010E3F6E84DF9DDF020E306E6C
:1003800044DF22EF05F03F6A7CDF95DF020E3F6E0F
:1003900078DF91DF020E306E38DF23EF05F033385F
:1003A000006E0F0E001600500F0B356E33500F0B02
:1003B000346E35C53FF565DF7EDFD50E006E002E4D
:1003C000FED734C53FF55DDF76DFD50E006E002E1B
:1003D000FED704EF02F03050000A07E0010A06E001
:1003E000030A07E0010A08E00AD009D0400E2F26D0
:1003F00006D0140E2F2603D0540E2F2600D0800EC8
:100400002F24326E336ECBD712003C383D6E0F0E68
:100410003D163C16100E3D243E6E3F6E32DF4BDF24
:10042000100E3C243E6E3F6E2CDF45DFD50E006E75
:10043000002EFED712000900F55210E0F6C42FF589
:10044000F7C430F5F8C431F5F5C43CF5DEDF2FC54F
:10045000F6F430C5F7F431C5F8F4EDD712002F6A81
:10046000306AB9DF880EF66E010EF76E000EF86E78
:10047000E2DF215242E12F6A010E306EACDF2250E2
:100480000BE0010A11E0030A17E0010A1DE0070A68
:1004900023E0010A29E030D0920EF66E010EF76ECD
:1004A000000EF86EC8DF28D09C0EF66E010EF76EB7
:1004B000000EF86EC0DF20D0A60EF66E010EF76EAD
:1004C000000EF86EB8DF18D0B00EF66E010EF76EA3
:1004D000000EF86EB0DF10D0BA0EF66E010EF76E99
:1004E000000EF86EA8DF08D0C40EF66E010EF76E8F
:1004F000000EF86EA0DF00D0BCD7216A5CEF05F0DB
:100500000301F38100003590F3A1358035B004D0AC
:100510003590F3A13580FAD7F3B1FED7EBC337F5A9
:10052000EAC336F536C501F537C502F500011200FC
:100530000301EC6BD50E006E002EFED7326A316AD5
:10054000306A2F6A346A336A3450000810E30001BD
:10055000D7DF02C503F501502F2602503022000ECE
:1005600031223222332AD8B4342A0301EDD730C5E0
:100570002FF531C530F532C531F5326A0F0E301620
:10058000316A326A2FC501F530C502F500016AEF04
:1005900005F08E0E006E30C501F52FC502F5036A19
:1005A000015209E102C501F5026A080E005E01521E
:1005B00002E1006A08D0D89001BE04D002360136AC
:1005C0000006F9D7019E12003C50D8B471D0006EDD
:1005D0004050D8B46DD0002604E3810E002668E2B6
:1005E00004D07F0E005E64E363E03DC544F54150F6
:1005F000441A3D8E418E3F504302F4C446F53E50AE
:100600004202F4C403F5F3C445F54302F350462611
:10061000F4504522000E03223F504202F35046267A
:10062000F4504522000E026A032202223D5043028A
:10063000F3504526F4500322000E02223D504202A0
:10064000F3500326F4500222000E016A01223F50AB
:100650004102F3504526F4500322000E02220122EB
:100660003E504102F3500326F4500222000E0122B4
:100670003D504102F3500226F4500122002A01BEEF
:1006800005D045360336023601360006000E45AE6B
:100690000AD0032A02220122015005E1025003E19F
:1006A000035001E1002A44BE018E44AE019E04D0F5
:1006B000006A016A026A036A12003C50B6083C6E86
:1006C000036A3DC540F53D8ED8903D323E323F3203
:1006D00003320232013200323C2EF6D740AE0BD04C
:1006E000001E011E021E031E002AD8B4012AD8B41F
:1006F000022AD8B4032AECEF03F0D8B204D0050ED6
:10070000EA6E440EE96E006A016A026A036A446A8C
:10071000456A466A476A43504210411040102CE037
:10072000200E486ED8903C363D363E363F36443635
:100730004536463647364350475C08E14250465CF2
:1007400005E14150455C02E14050445C0FE34050FC
:10075000445E4150D8A0413C455E4250D8A0423C46
:10076000465E4350D8A0433C475ED88000360136F1
:1007700002360336482ED6D744C5EFF445C5ECF40F
:1007800046C5ECF447C5ECF41200E950346E335022
:10079000366E19E032C53FF531C53EF530C53DF541
:1007A0002FC53CF5436A426A200E416E820E406EB0
:1007B0000BDF03C532F502C531F501C530F500C5C3
:1007C0002FF5362EE7D732C53FF531C53EF530C59A
:1007D0003DF52FC53CF571D703C532F502C531F59E
:1007E00001C530F500C52FF532AE0DD03406348A80
:1007F0002F1E301E311E321E2F2AD8B4302AD8B4F4
:10080000312AD8B4322A3B0E3B6E9A0E3A6ECA0E8B
:10081000396E386A0A0E366E3350D8B4342AD8820C
:10082000050EEA6E2F0EE96E32C53FF531C53EF575
:1008300030C53DF52FC53CF53BC543F53AC542F5FE
:1008400039C541F538C540F558DF015000520FE178
:100850003328365C0CE034500CE00F0B365C01E0C2
:1008600037E234BE35D034BC04D0200E2DD0200E5B
:10087000341634AA0CD0349A3350D8A4340600501D
:10088000346E2D0E3C6EC1DD3450006E346A335030
:10089000365C0AE10050346E2E0E3C6EB6DD3450EC
:1008A000006E200E3416000E300E34AA0DD0349A8D
:1008B0003350D8A434060050346E2D0E3C6EA5DDA6
:1008C0003450006E346A300E002600C53CF59DDDC4
:1008D000D8923BC53FF53AC53EF539C53DF538C51B
:1008E0003CF5436A426A416A0A0E406E06DF03C560
:1008F0003BF502C53AF501C539F500C538F5362E88
:100900008ED71200010E0301EC6FD50E006E002E83
:10091000FED7326A316A306A2F6A346A336A3450D9
:1009200000081DE31C520DE01D52D8B4FDD7000194
:10093000E7DD01502F2602503022000E31223222F4
:1009400009D00001DDDD01502F2602503022000EBB
:1009500031223222332AD8B4342A0301E0D730C5F9
:100960002FF531C530F532C531F5326A0F0E30162C
:10097000316A326A2FC501F530C502F50001C0EFBA
:1009800005F00900F6C430F5F7C431F5F8C432F5C6
:10099000F5C43CF53ADD30C5F6F431C5F7F432C59F
:1009A000F8F42F2EEED71200F86AD69A078EB06BA5
:1009B000AF6BB36B080EB16F600EAD6F1B6A1C6A34
:1009C0001D6A1F6A1E6A206A216A226A236A286ACF
:1009D000276A0401006B086B106B206B0001716BC0
:1009E000726B736B706B756B766B776B746B010EE0
:1009F000246E256E266AB06BAF6BB36B030EB16FBE
:100A0000600EAD6F280E306E00DCB06BAF6BB36B59
:100A1000050EB16F600EAD6F280E306E05EC01F063
:100A2000B06BAF6BB36B080EB16F600EAD6F280E7D
:100A3000306E05EC01F01AEF01F0640E306E05EC3B
:100A400001F03ED4A0D42F6A306AC5DCCE0EF66E1B
:100A5000010EF76E000EF86EEEDC2F6A010E306E9E
:100A6000BADCD80EF66E010EF76E000EF86EE3DCFF
:100A7000080E2F6EFA0E306E05EC01F02F2EFAD70D
:100A8000800E03011A6F450E1B6F1AA901D0196B56
:100A9000070E186FA18EC00ED612236A20520FE0E7
:100AA0001C5202E01C6A02D0010E1C6E216A010E6B
:100AB000236E206A0001D3D4216A236A03012152E4
:100AC00007E01C5202E01C6A02D0010E1C6E216A73
:100AD00000012ED502C52EF501C52DF52F6A306A0D
:100AE0007ADC2D3C03D02E500F083AE02EC530F5AD
:100AF0002DC52FF54EDD03C52CF502C52BF501C51F
:100B00002AF500C529F52CC53FF52BC53EF52AC5AC
:100B10003DF529C53CF5B10E436E470E426E7A0E87
:100B2000416E760E406E50DD03C52CF502C52BF5E7
:100B300001C52AF500C529F5050EE96E2CC532F56B
:100B40002BC531F52AC530F529C52FF5030E336EB7
:100B50001CDE560E3C6E59DC200E3C6E56DC07D077
:100B6000E20EF66E010EF76E000EF86E64DC2F6A70
:100B7000010E306E30DC1C5251E01BC57DF0C2D638
:100B800002C52EF501C52DF52D3C03D02E500F08C2
:100B90003DE02EC530F52DC52FF5FBDC03C52CF54A
:100BA00002C52BF501C52AF500C529F52CC53FF571
:100BB0002BC53EF52AC53DF529C53CF5F60E436E1D
:100BC000CF0E426E530E416E730E406EFDDC03C5B8
:100BD0002CF502C52BF501C52AF500C529F5040E33
:100BE000E96E2CC532F52BC531F52AC530F529C57E
:100BF0002FF5030E336EC9DDF10EF66E010EF76EA2
:100C0000000EF86E030E2F6EBCDE07D0F60EF66EE9
:100C1000010EF76E000EF86E0EDC3CD07D6B306A74
:100C20001BC52FF5B6DC03C52CF502C52BF501C598
:100C30002AF500C529F52CC53FF52BC53EF52AC57B
:100C40003DF529C53CF5A10E436EA00E426E200E67
:100C5000416E770E406EB8DC03C52CF502C52BF54E
:100C600001C52AF500C529F5030EE96E2CC532F53C
:100C70002BC531F52AC530F529C52FF5020E336E87
:100C800084DD050EF66E020EF76E000EF86E040E91
:0A0C90002F6E77DE030102D7030088
:020000040030CA
:0A0000008CFF36DF9FFFFFFFFFFFBC
:00000001FF
